:020000020000FC
:1000000015C0189518951895189553C118951895F9
:1000100018951895189518951895189518950F8096
:10002000F00000000030010624BC6A000FE50DBF9F
:1000300002E00EBF00E207B907EE06B9C49ABC9A07
:10004000B898B998C098C19800E806BD03E006BD0D
:1000500002E003BF02E009BFBA9ABC9AC298C098F6
:10006000F0E0EEE1259035904590559065907590C3
:10007000F0E0E6E285909590A590B59078944AEFEF
:1000800015D13AD0C5D0F2E0EAED10E8D0D0EBD0EF
:100090004AEF0CD130E00FD02317E9F318F015D058
:1000A000339502C01CD03A9567D0B49A10ECBFD0FB
:1000B000022FECD0F1CF0F9303E207B90F91369ADC
:1000C000349BFECF349A25B1089500277B0C6A1C1F
:1000D000591C481C301E201E00EF402A089500279E
:1000E0000FE0402200277B186A0859084808300AA8
:1000F000200A00EF402A089563E07FEF4DD060E1D1
:1001000070E84AD061E170E847D062E170E844D01D
:1001100065E970E041D06AE270E03ED06BE271E0E8
:100120003BD06FE270E038D060E370E035D061E33F
:1001300070E032D060E17FE42FD061EB70EA2CD028
:1001400063E07EEF29D06AE17FEF26D06BE17FEF9D
:1001500023D06CE170E020D00FD0F0E0E4E26CE25C
:1001600075911AD06DE2759117D06EE270E014D0DF
:1001700061EB70E211D008956DE1722D0DD06EE14A
:10018000732D0AD06FE1742D07D060E2752D04D075
:1001900061E2762D01D0089506D0562F09D0572F51
:1001A00007D023D0089550ECB89A28D0B99A26D019
:1001B0000894551F59F010F4B89801C0B89A20D08F
:1001C000B9981ED0B99A1CD0550FF4CFB89818D052
:1001D000B99816D0B19BFECFB89A12D0B99A10D068
:1001E0008894B09908940AD00895B99AB89A08D01A
:1001F000B99806D0B89804D00895089503E001C0D6
:1002000002E01FB71F930A95F1F71F911FBF0895D2
:1002100044E14CD018E30BD042E048D01EE007D0B8
:1002200042E044D011E003D042E040D008950F9363
:10023000012F0BD0C49803C00F9307D0C49AC29A61
:1002400042E0C29833D00F9108950F931F9318E0A6
:10025000C498000F08F4C49AB89AB8981A95C1F7D0
:100260001F910F9108950591002311F0E5DFFBCF59
:10027000B0E0A0E61C91143020F01395183008F07F
:1002800013950BE8011B102FD2DF08950F930295F1
:1002900003D00F9101D008951F930F7000630A33AC
:1002A00010F017E0010FC8DF1F9108954423F1F704
:1002B00008950F931F930FB70F9303E802BF4423D2
:1002C00009F04A950F910FBF1F910F9118950F9349
:1002D0000FB7B49A0FBF0F911895202041534D20AE
:1002E0005475746F7269616C2020000020202020FA
:1002F00020526561647921202020202000002020E8
:1003000020202020204F4B212020202020200000D2
:00000001FF
